:02000000AC282A
:100008008C00030E83018E000A088D0077282C08C7
:100018002106BE00AC1F1528AC09AE09AE0F152885
:10002800AC0AA11F1C28A109AD09AD0F1C28A10A03
:100038002A20BE1F0800BE00BE09A009BE0F252841
:10004800A00A3E0808009030BD002C281030BD00E2
:10005800C001A0012C0DC00DA00D2D08C002210863
:10006800031C210FA002031840282D08C0072108EF
:100078000318210FA0070310AE0DAC0DBD031F30F0
:100088003D05031D2E28BD1B4D282C08A0002E0859
:100098000800400808001030BE00A001BD01AC0CEB
:1000A800AE0C031C5D282D08BD070318A00A210803
:1000B800A0070310AD0DA10DBE0B53283D08080085
:1000C800430803197628C201FF3042028F01031C3E
:1000D8008F0A0F0803197328C20A42036828C3034A
:1000E800430A642808000B113708B60A0319B70A2F
:1000F80035303602A3003708A400031CA4030C30D3
:10010800A402A201A41FA20A22080319A428B60166
:10011800B7010130CF003B08BA0A0319BB0AE03027
:100128003A02A3003B08A400031CA4030130A40264
:10013800A501A41FA50A25080319A428BA01BB0113
:1001480083010D088A000E0E83008C0E0C0E090028
:100158008316B601B701B301B40101308100FF3045
:10016800850086018312860181018B1603118B1786
:10017800B001073030028F0090018F1B900A1008E1
:100188000319CE283008263E831384008001B00A64
:100198003003BD28B0010530300291009201911B57
:1001A800920A12080319D32B83120508C1004108CB
:1001B800073C94009501941B950A150891000319B2
:1001C800EE2804303002940095011408031D950AA6
:1001D8001508910011080319692A3A08AE003B086E
:1001E800AC000830AD00A101272097002008980036
:1001F8001708BC00B5013C080319B50A3508950075
:10020800031D0F2901303C02B500BF013508031951
:10021800BF0A3F08950015089400031D1C290230E9
:100228003C029500B50115080319B50A3508940074
:100238001408031978293008AF0000302F02031979
:10024800322901302F020319402902302F020319E5
:10025800522903302F020319652977292608AE0091
:10026800AC011030AD00A1014F20970020089E007E
:100278009B0017089A0077292708AE00AC011030B8
:10028800AD00A1014F20970020089800970A031895
:10029800980A18089B0017089A0077292A08AE00C0
:1002A800AC011030AD00A1014F20970020089E003E
:1002B8000230970703189E0A1E089B0017089A0029
:1002C80077292B08AE00AC011030AD00A1014F20FA
:1002D800970020089800033097070318980A180811
:1002E8009B0017089A00642A03303C029500B50168
:1002F80015080319B50A35080319DB293008AF00BA
:1003080000302F020319952901302F020319A32960
:1003180002302F020319B52903302F020319C82907
:10032800DA292608AE00AC011030AD00A1014F203B
:10033800970020089E009B0017089A00DA292708D2
:10034800AE00AC011030AD00A1014F20970020088D
:100358009800970A0318980A18089B0017089A002B
:10036800DA292908AE00AC011030AD00A1014F20F8
:10037800970020089E000230970703189E0A1E085F
:100388009B0017089A00DA292A08AE00AC01103041
:10039800AD00A1014F20970020089800033097076F
:1003A8000318980A18089B0017089A00642A043052
:1003B8003C02B8009C01380803199C0A1C08B900C3
:1003C800031DEF2905303C02B8009C0138080319C9
:1003D8009C0A1C08B9003908BF00031DFC29063017
:1003E8003C02B900B80139080319B80A3808BF0037
:1003F8003F089500031D092A07303C02BF00B901D8
:100408003F080319B90A3908950015080319642A21
:100418003008AF0000302F0203191F2A01302F02C5
:1004280003192D2A02302F0203193F2A03302F0205
:100438000319522A642A2608AE00AC011030AD0018
:10044800A1014F20970020089E009B0017089A00E2
:10045800642A2708AE00AC011030AD00A1014F207E
:10046800970020089800970A0318980A18089B0014
:1004780017089A00642A2808AE00AC011030AD00B5
:10048800A1014F20970020089E000230970703180B
:100498009E0A1E089B0017089A00642A2908AE00C5
:1004A800AC011030AD00A1014F2097002008980042
:1004B800033097070318980A18089B0017089A0032
:1004C800083041029500C100862A023030079500A5
:1004D8001508263E831384000008AE00AC011030D6
:1004E800AD00A1014F20970020089E003008970713
:1004F80003189E0A0001B01BFF309E071E089B00D0
:1005080017089A0083121A08860004303002B900CE
:10051800B8013908031DB80A380803199A2A0430A3
:10052800C30064208312FF3086000A2B3608AE0011
:100538003708AC000430AD00A1010B20970020085B
:100548009800B2001708B1003108093C9700023042
:100558009E00031C9E0332089E029C019E1B9C0A5F
:100568001C080319C52A87303102970032089E00FB
:10057800031C9E0301309E021E08B2001708B1003A
:10058800D22A3108093C970002309800031C9803CE
:10059800320898021808B2001708B10001309A0012
:1005A8009B0131081A0297001B089E00031C9E033A
:1005B80032089E029F019E1B9F0A1F080319E82A02
:1005C8009A0FD52A9B0AD52A8312FF30860001305C
:1005D8009A009B013108123C970004309E00031CCE
:1005E8009E0332089E0217081A0297001B089800FB
:1005F800031C98031E0898029301981B930A13087A
:1006080003190A2B9A0FEE2A9B0AEE2ACE014F08ED
:10061800031DCE0A4E0803195F2BCF01A60A260830
:10062800093CCD01031CCD0A4D0803191E2BA60158
:10063800A70A27032708053CCC01031CCC0A4C0851
:100648000319292BA701A80A28032808093CCB016C
:10065800031CCB0A4B080319342BA801A90A290348
:100668002908053CCA01031CCA0A4A0803193F2B7A
:10067800A901AA0A2A032A08093CC901031CC90AB4
:10068800490803194A2BAA01AB0A2B032B08013C82
:10069800A001031CA00A2008C80003195A2B2A0825
:1006A800033CA001031CA00A2008C800480803193D
:1006B8005F2BAA01AB014108AF0003302F020319D9
:1006C8006E2B05302F020319712B06302F020319E8
:1006D8009B2BD02BA601A701D02B3408B30A0319F2
:1006E800B40A3308643C97009801031C9803340843
:1006F80098029601981B960A160803199A2BB301BB
:10070800B401A80A2808093CC701031CC70A4708FE
:100718000319912BA801A90A29032908053CC60138
:10072800031CC60A460803199A2BA901D02B3408C2
:10073800B30A0319B40A3308643C97009801031CF0
:100748009803340898029901981B990A1908031903
:10075800D02BB301B401AA0A2A08093CC501031C1D
:10076800C50A45080319BB2BAA01AB0A2B032B08A2
:10077800013CA001031CA00A2008C4000319CB2BCC
:100788002A08033CA001031CA00A2008C40044084E
:100798000319D02BAA01AB01B00A3003CF28CE2809
:0207A800D42B50
:02400E00FA3F77
:00000001FF
